:020000040000FA
:02000000ED2BE6
:10028C00003414346434FF34043464008001840A70
:10029C0004060319003404064C2900000000000079
:1002AC00000000000000000000000800F601F11F33
:1002BC00602961296829F009F109F00A0319F10A8A
:1002CC00F601F60AF31F6B296C297529F209F3095B
:1002DC00F20A0319F30A0130F4007408F606F70168
:1002EC00F8017008710403197C297D29B429F501E2
:1002FC00F50A8B2901300310F00DF10DFF3E031DA3
:10030C0081290130F4007408F507F11F8E298F291B
:10031C00802901300310F70DF80DFF3E031D9029C5
:10032C0071087302031D9C2970087202031C9F291B
:10033C00A029A7297008F2027108031CF303F30229
:10034C00771401300310F10CF00CFF3E031DA829AB
:10035C000130F502031DB329B4298F29760803193E
:10036C00B829B929BE29F709F809F70A0319F80AB7
:10037C007808F1007708F000080083160313860153
:10038C00FB018312AE01AF01FC01FD0183160313C7
:10039C0086138312031386175321831603138617B0
:1003AC00DD290130FC070318FD0A0030FD0783121C
:1003BC00861BE129E229D7291030F0000030F1002A
:1003CC007D08F3007C08F2005C2170088312031393
:1003DC00AE070318AF0A7108AF07AC01AD01FC0101
:1003EC00FD018316031306138312031306175321FF
:1003FC00831603130617082A0130FC070318FD0A9D
:10040C000030FD078312061B0C2A0D2A022A10301D
:10041C00F0000030F1007D08F3007C08F2005C2154
:10042C00700883120313AC070318AD0A7108AD07EB
:10043C00AA01AB01FC01FD01831603138612831282
:10044C00031386165321831603138616332A0130A1
:10045C00FC070318FD0A0030FD078312861A372AA1
:10046C00382A2D2A1030F0000030F1007D08F300FE
:10047C007C08F2005C21700883120313AA0703188E
:10048C00AB0A7108AB07A801A901FC01FD01831699
:10049C000313061283120313061653218316031338
:1004AC0006165E2A0130FC070318FD0A0030FD0712
:1004BC008312061A622A632A582A1030F000003080
:1004CC00F1007D08F3007C08F2005C2170088312B7
:1004DC000313A8070318A90A7108A9070130F9002A
:1004EC007908FB0710307B02031C7D2A7E2AC72962
:1004FC000F30F9007908B4000F30F9007908B30017
:10050C000F30F9007908B2000F30F9007908B1000A
:10051C00FF308316031392000430831203139200EE
:10052C000C3097003008353E84008313000895008A
:10053C00FC01FD0183160313861383120313861724
:10054C005321831603138617B12A0130FC070318B5
:10055C00FD0A0030FD078312861BB52AB62AAB2A8A
:10056C002E087C02F9002F08031C2F0A7D02FA00CA
:10057C007A08803A803C031DC52A79083402031896
:10058C00C82AC92AD12A143083120313A6000030BA
:10059C00A7000614EC2A831203132708803AFF00E5
:1005AC0080307F02031DDC2A01302602031CDF2A67
:1005BC00E02AE92AFF3083120313A6070318A70ABF
:1005CC00FF30A707EC2A831203130610FC01FD0170
:1005DC008316031306138312031306175321831672
:1005EC0003130617FF2A0130FC070318FD0A00301D
:1005FC00FD078312061B032B042BF92A2C087C0203
:10060C00F9002D08031C2D0A7D02FA007A08803AA5
:10061C00803C031D132B790833020318162B172B60
:10062C00262B8312031324082504031D1E2B1F2BBA
:10063C00212B023086061430A4000030A5003D2B7F
:10064C00831203132508803AFF0080307F02031DBC
:10065C00312B01302402031C342B352B3D2BFF3066
:10066C0083120313A4070318A50AFF30A507FC0186
:10067C00FD0183160313861283120313861653216E
:10068C00831603138616502B0130FC070318FD0A42
:10069C000030FD078312861A542B552B4A2B2A083F
:1006AC007C02F9002B08031C2B0A7D02FA007A0845
:1006BC00803A803C031D642B790832020318672BA7
:1006CC00682B702BF43083120313A2000130A300AB
:1006DC0006158B2B831203132308803AFF008030FE
:1006EC007F02031D7B2B01302202031C7E2B7F2BF0
:1006FC00882BFF3083120313A2070318A30AFF30C1
:10070C00A3078B2B831203130611FC01FD01831627
:10071C0003130612831203130616532183160313B5
:10072C0006169E2B0130FC070318FD0A0030FD074E
:10073C008312061AA22BA32B982B28087C02F900F3
:10074C002908031C290A7D02FA007A08803A803CA9
:10075C00031DB22B790831020318B52BB62BD42B01
:10076C008312031320082104031DBD2BBE2BCF2B9A
:10077C000130F9007908B00704303002031CC72B94
:10078C00C82BC92BB0013008353E840083130008F8
:10079C0095001430A0000030A1009E2A8312031390
:1007AC002108803AFF0080307F02031DDF2B0130CF
:1007BC002002031CE22BE32B9E2AFF30831203132F
:1007CC00A0070318A10AFF30A1079E2A0028462182
:1007DC00B5004721B6004821B7004921B8004A218D
:1007EC00B90083132030840035304B21FC01FD010E
:0407FC008301C32989
:02400E0058FF59
:00000001FF
